:020000040000FA
:02000000BC2E14
:08000800FF000308FE000A08D6
:10001000FC000408FD008312031300308A00233023
:100020008100A10A103021020318A1012014A20F9F
:100030001C28A30F1C28A0143D08003E03193628D5
:100040002E1C342887018714142301301E2300003E
:100050001E30A400871007301E23871406301E238D
:10006000A40B2A2887107E28142338280923052367
:100070000A30A500AB21B121BF210D238501210844
:100080000319892001302102031996200230210230
:100090000319A320033021020319B02004302102E8
:1000A0000319BD20053021020319CA2006302102A0
:1000B0000319D720073021020319E4200830210258
:1000C0000319F120093021020319FE200A30210210
:1000D00003190B210B302102031918210C302102C6
:1000E000031925210D302102031932210E3021027E
:1000F00003193F210F30210203194C210B118B17DB
:100100007D0884007C088A007E088300FF0E7F0E35
:10011000090000308700B030840083138221303022
:10012000840083175921A50B8B2808000130870014
:10013000D030840083138221B0308400831759218A
:10014000A50B9828080020308700B830840083135E
:1001500082213830840083175921A50BA528080077
:1001600021308700D830840083138221B830840086
:1001700083175921A50BB228080040308700C030F2
:100180008400831382214030840083175921A50BFA
:10019000BF28080041308700E030840083138221AB
:1001A000C030840083175921A50BCC28080060308B
:1001B0008700C8308400831382214830840083176D
:1001C0005921A50BD928080061308700E830840048
:1001D00083138221C830840083175921A50BE62898
:1001E000080080308700103084008317822150304F
:1001F000840083175921A50BF3280800813087005C
:100200009030840083178221D030840083175921D5
:10021000A50B00290800A030870018308400831740
:1002200082215830840083175921A50B0D2908001D
:10023000A13087009830840083178221D830840051
:1002400083175921A50B1A290800C03087002030D8
:100250008400831782216030840083175921A50B05
:1002600027290800C1308700A0308400831782212D
:10027000E030840083175921A50B34290800E030B1
:100280008700283084008317822168308400831718
:100290005921A50B41290800E1308700A8308400CE
:1002A00083178221E830840083175921A50B4E293A
:1002B000080085010108000203180514840A0108DA
:1002C000000203188514840A0108000203180515AA
:1002D000840A0108000203188515840A0108000237
:1002E00003180516840A0108000203188516840AFB
:1002F0000108000203180517840A01080002031808
:100300008517080086010108000203180614840AF4
:100310000108000203188614840A01080002031869
:100320000615840A0108000203188615840A0108CC
:10033000000203180616840A010800020318861634
:10034000840A0108000203180617840A0108000243
:100350000318861708000310260DAF00B821B2005D
:1003600008000310260D013EAF00B821B3000800BD
:1003700001308A002F08C33E03188A0A820032081F
:100380008A00330882000234033402340E3402340B
:10039000163402341E340234263402342E3402342D
:1003A0003634023442340234463402345234023495
:1003B0005634023462340234663402347234023405
:1003C0007634023482340234863402349234023475
:1003D00096340234A2340234A6340234B2340234E5
:1003E000B6340234C2340234C6340234D234023455
:1003F000D6340234E2340234E6340234F2340234C5
:10040000F634033402342D103030B10028180B2A92
:100410000630A600042B0130A600042B2818132A4E
:100420000030A600042B0230A600042B28181B2A3B
:100430000030A600042B0330A600042B2818232A22
:100440000430A600042B0330A600042B28182B2A06
:100450000030A600042B0530A600042B2818332AF0
:100460000730A600042B0030A600042B2818402AD1
:100470000030310703193E2AB10B042B2D14042B35
:10048000A601042B2808AC00A60A042B2C08280679
:10049000031D4C2AA601042B28182B10281C2B14F2
:1004A000A60A042B2808AC00A60A042B2C08280650
:1004B000031D5C2AA601042B28182A12281C2A16C0
:1004C000A60A042B2808AC00A60A042B2C08280630
:1004D000031D6C2AA601042B2818AA11281CAA1592
:1004E000A60A042B2808AC00A60A042B2C08280610
:1004F000031D7C2AA601042B28182A11281C2A1562
:10050000A60A042B2808AC00A60A042B2C082806EF
:10051000031D8C2AA601042B2818AA10281CAA1433
:10052000A60A042B2808AC00A60A042B2C082806CF
:10053000031D9C2AA601042B28182A10281C2A1403
:10054000A60A042B2808AC00A60A042B2C082806AF
:10055000031DAC2AA601042B2818A912281CA916D1
:10056000A60A042B2808AC00A60A042B2C0828068F
:10057000031DBC2AA601042B28182912281C2916A1
:10058000A60A042B2808AC00A60A042B2C0828066F
:10059000031DCC2AA601042B2818A911281CA91573
:1005A000A60A042B2808AC00A60A042B2C0828064F
:1005B000031DDC2AA601042B28182911281C291543
:1005C000A60A042B2808AC00A60A042B2C0828062F
:1005D000031DEC2AA601042B2818A910281CA91415
:1005E000A60A042B2808AC00A60A042B2C0828060F
:1005F000031DFC2AA601042B28182910281C2914E5
:10060000A60A042BA60130140800AD10071DAD1476
:100610000800281089192814080027082602031C3E
:10062000132B2608A70008002E10BD030310BC0CD6
:10063000BB0CBA0CB90C03182E140800B400B40B90
:100640001F2B0800BA01BB01BC01A030B900B709DB
:10065000371C3A143718BA14351E3A15351ABA151C
:10066000B51D3A16B519BA16351D3A173519BA1708
:10067000B51C3B14B518BB14351C3B153518BB1500
:10068000B61E3B16B61ABB16361E3B17361ABB17DC
:10069000B61D3C14B619BC14361D3C153619BC15D4
:1006A000B61C3C16B618BC16361C3C173618BC17C0
:1006B0002130BD000800BE01BF010830C00003109A
:1006C000C20CBF0DBE0DC10CBF0DBE0DC00B5F2B0C
:1006D0000800C3000000C30B6A2B0800CD0A4D08B8
:1006E000133C0319CD014D08B800FB01FA010800C5
:1006F000CD034D08013E031D802B1230CD00B80004
:10070000FB01FA0108002908CD00B800ED3E031CEA
:100710008D2B1230CD024D08862BFB01FA0108000B
:10072000C4002010201C922BC40B912B08004F30CA
:10073000840083132030C7008001840AC70B9C2BE0
:10074000C5014D0AC6000A304602031CAB2B0A3015
:10075000C602C50AA32B1030C607C507711CB52BEE
:100760004F30840083132430C32355308400831317
:100770004508C323840A83134608C323FF300F268A
:10078000FF300F260800BE004A30F6001730F50093
:100790003E0803103E0DF6070318F50A0310BE0DC0
:1007A000BE0D0318F50A3E08F6070318F50A8B1369
:1007B0001427C1004B088A008B170130F607031875
:1007C000F50A8B131427C0004B088A008B174008CA
:1007D0008000840A0130F6070318F50AC10BE12BEB
:1007E00008000730C8001A30C90003104D0DFB0087
:1007F0008B130D278B17CA0003144D0DFB008B13B1
:100800000D278B17C9004A08C8000800213048028C
:10081000031D0E2C49087B073B24202C8B130A0850
:10082000CB0048087A07F500031049087B07F6005B
:100830000318F50A1427CC004B088A004C088B17C4
:10084000FB0F232CFA0A0800831603178C18262C9A
:100850008B130C15831203177B088D0079088C000D
:100860008316031755308D00AA308D008C148B171A
:100870008312031308008B13831603178C183E2C66
:100880000C11831203178D00831603178C130C149D
:10089000831203170C08831203138B17080001300F
:1008A0003B24F10008004F24711C582C7110592C66
:1008B00071140130FB007108F90024249723972359
:1008C0000800F123FB01FA010624CE00CE13062412
:1008D000F000F00A0624F200301C8A2C07302A02AD
:1008E000031D752C8323B001612CAA08031D8A2CDB
:1008F0002030290203196E2321302902031978239D
:10090000003029020319CD010C30290203195324A8
:10091000B001612C2D080319A02C972397230330D5
:100920002D02031953242D18982CAD189C2C612CE2
:100930006E23972397238F2C7823972397238F2C2D
:100940000C304E020319E12416304E0204308A00A6
:100950000319F22404308A0018304E0205308A0050
:100960000319122504308A0019304E0205308A001E
:100970000319242504308A001A304E0205308A00FB
:1009800003197E2D04308A003D08003E031DD42C3F
:10099000A01CD42CA010711CCF2C6E23612C07300E
:1009A000B5003808B6002223F20B6C2C612C730DB5
:1009B000730D731A013AF31A013AF319013AF3006D
:1009C00008004F30840083132030BE00D724D72482
:1009D000D724D724D7248000840ABE0BE62C7008C5
:1009E0000F2608004F30840083132030F4000624C3
:1009F0008000840AF40BF72C70080F2670080F266D
:100A000070080F2670080F2608004F3084008313EB
:100A10001F30F400840A000884038000840AF40B69
:100A20000A2D080005255E308400062480006E3003
:100A300084000624800070080F2670080F267008B6
:100A40000F2670080F2608000624BE00BE082030BE
:100A50003E0203182E2D3E08BF007D2D2030BE0221
:100A60004A30F6001730F5003E0803103E0DF60739
:100A70000318F50A0310BE0DBE0D0318F50A3E0853
:100A8000F6070318F50A8B131427C1004B088A00D8
:100A90008B170130F6070318F50A8B131427C000D3
:100AA0004B088A008B1705254008EE004008DE0041
:100AB0003F1CEE013F1DDE01BF18EE09BF19DE0924
:100AC0000130F6070318F50A70080F2670080F2684
:100AD00070080F2670080F26C10B4D2D0525EE015D
:100AE000DE01BF18EE09BF19DE0970080F26700875
:100AF0000F2670080F2670080F260800EF004F30F1
:100B0000840083132030BF0006248000840ABF0BBA
:100B1000842D6430BF00B030840083134F08DD257E
:100B20005008DD255108DD255208DD2510308400F0
:100B300083175308DD255408DD255508DD255608A3
:100B4000DD255708DD255808DD255908DD255A081B
:100B5000DD255B08DD255C08DD255D08DD255E08FB
:100B6000DD25D030840083135F08DD256008DD2596
:100B70006108DD256208DD25903084008317630855
:100B8000DD256408DD256508DD256608DD256708A7
:100B9000DD256808DD256908DD256A08DD256B0887
:100BA000DD256C08DD256D08DD256E08DD256F0867
:100BB0009023BF0B8B2D8313C42CBE00BE1B0726B6
:100BC000BE1F0B26840A3E1B07263E1F0B26840AE7
:100BD000BE1A0726BE1E0B26840A3E1A07263E1E94
:100BE0000B26840ABE190726BE1D0B26840A3E1951
:100BF00007263E1D0B26840ABE180726BE1C0B26A0
:100C0000840A3E1807263E1C0B26840A0800800A28
:100C10000319800908008008031D80030800EF0005
:100C2000B030840083134F086026500860265108B6
:100C3000602652086026103084008317530860260F
:100C40005408602655086026560860265708602616
:100C500058086026590860265A0860265B086026F6
:100C60005C0860265D0860265E086026D03084003F
:100C700083135F08602660086026610860266208AA
:100C8000602690308400831763086026640860261D
:100C90006508602666086026670860266808602682
:100CA000690860266A0860266B0860266C08602662
:100CB0006D0860266E0860266F0890238313080075
:100CC000F4008001F41B8009840A8001741B8009F0
:100CD000840A8001F41A8009840A8001741A800948
:100CE000840A8001F4198009840A8001741980093A
:100CF000840A8001F4188009840A8001741880092C
:100D0000840A080002302602031C0301CF000030D1
:100D1000D00001300F262D080319A02EA701A6012F
:100D20003D08003E031D8B2E2D08D000CF012D085D
:100D3000D20001300F26B5010C30B60022238B2ED5
:100D4000301C822EB001F030CF00D0017F300F2652
:100D5000CF01D0013F300F26F030CF00D0017F30DF
:100D60000F262908CF002A08D000FF300F26FF30B9
:100D70000F26A701A601822E85018101CD01BD01AB
:100D8000AB01AA01A901AC01A601A701B001A10113
:100D9000A201A301AD018316031371308F048316E2
:100DA000031788018901831603138230810083169B
:100DB00003131C30870085018601083089008312E7
:100DC0000313AD011D30F3008B168B174F308400D9
:100DD0002030F400FF308000840AF40BEB2EFF304B
:100DE0000F26FF300F264F3084002030F4000030F3
:100DF0008000840AF40BF82EFF300F26FF300F26F8
:100E0000FF300F264F242D08D000FF300F26FF3073
:100E10000F262D1C612C5324822E48088A007B0843
:100E2000490703188A0A82000A08CB0075088A005D
:100E3000760882000734403407345334073456347C
:100E400007348F340734C7340734F1340834093495
:100E500008342434083465340E34683410346B3468
:100E60001034AE34113451341134D4341234D734F4
:100E700013345A3414345D341634A0341734033424
:100E800019340F3410340534203420344434013400
:100E9000553443344B344F344E34043431343834C5
:100EA0002034203420340C343F34003419340F34CF
:100EB00036340134203420344434753463346B3494
:100EC0006F346E3420343134383420342D342034AF
:100ED0000534323430343034393420344134203421
:100EE0004434753463346B3420344F3464346434A4
:100EF0006934743479342034203420344A347534DD
:100F00006E3465342034313432342D343134343459
:100F100020343234303430343934203420341934ED
:100F20000F343534043420342034493420347734B9
:100F300065346E347434203474346F342034443463
:100F4000753463346B346F346E3431343834203458
:100F500061346E34643420346234753469346C34F2
:100F60007434203474346834693473342034053470
:100F700063346F346F346C342034013462346C3435
:100F800069346E346B346934653420342034193458
:100F90000F34273401342034203473346F34203438
:100FA0006D3461346E347934203462346C34693495
:100FB0006E346B346934653473342C342034043427
:100FC00073346F3420346C346934743474346C3456
:100FD00065342034743469346D3465342E342034EF
:100FE000203419340F34153401342034203477344C
:100FF000773477342E340434323464346B346934C7
:101000007434733401342E3463346F346D342034CB
:10101000203419340F34183401342034203444344B
:10102000753463346B346F346E3431343834043493
:10103000203442346C3469346E346B346934653432
:10104000733421342034203418340F341F340134E5
:10105000003403340034073400340F3400341F34B8
:1010600000343F3400347F340034FF3400347F34A4
:1010700080343F34C0341F34E0340F34F03407344C
:10108000F8340334FC340134FE340034FF340134CA
:10109000FF340334FF340734FF340F34FF341F347C
:1010A000FF343F34FF347F34FF34FF34FF347F3468
:1010B0007F343F343F341F341F340F340F34073430
:1010C0000734033403340134013416341F3430340C
:1010D000FF34003400340034003400340034003471
:1010E0000034003400340034003400340034003460
:1010F0000034003400340034003400340034003450
:10110000003400340034003400340034003400343F
:101110000034FF3400340034003400340034003430
:10112000003400340034003400340034003400341F
:10113000003400340034003400340034003400340F
:1011400000340034003400340034003400340034FF
:1011500000340034FF3400340034003400340034F0
:1011600000340034003400340034003400340034DF
:1011700000340034003400340034003400340034CF
:1011800000340034003400340034003400340034BF
:10119000003400340034FF340034003400340034B0
:1011A000003400340034003400340034003400349F
:1011B000003400340034003400340034003400348F
:1011C000003400340034003400340034003400347F
:1011D0000034003400340034FF3400340034003470
:1011E000003400340034003400340034003400345F
:1011F000003400340034003400340034003400344F
:10120000003400340034003400340034003400343E
:1012100000340034003400340034FF34003400342F
:10122000003400340034003400340034003400341E
:10123000003400340034003400340034003400340E
:1012400000340034003400340034003400340034FE
:10125000003400340034003400340034FF340034EF
:1012600000340034003400340034003400340034DE
:1012700000340034003400340034003400340034CE
:1012800000340034003400340034003400340034BE
:101290000034003400340034003400340034FF34AF
:1012A000003400340034003400340034003400349E
:1012B000003400340034003400340034003400348E
:1012C000003400340034003400340034003400347E
:1012D000003400340034003400340034003400346E
:1012E000FF3400340034003400340034003400345F
:1012F000003400340034003400340034003400344E
:10130000003400340034003400340034003400343D
:10131000003400340034003400340034003400342D
:101320000034FF340034003400340034003400341E
:10133000003400340034003400340034003400340D
:1013400000340034003400340034003400340034FD
:1013500000340034003400340034003400340034ED
:1013600000340034FF3400340034003400340034DE
:1013700000340034003400340034003400340034CD
:1013800000340034003400340034003400340034BD
:1013900000340034003400340034003400340034AD
:1013A000003400340034FF3400340034003400349E
:1013B000003400340034003400340034003400348D
:1013C000003400340034003400340034003400347D
:1013D000003400340034003400340034003400346D
:1013E0000034003400340034FF340034003400345E
:1013F000003400340034003400340034003400344D
:10140000003400340034003400340034003400343C
:10141000003400340034003400340034003400342C
:1014200000340034003400340034FF34003400341D
:10143000003400340034003400340034003400340C
:1014400000340034003400340034003400340034FC
:1014500000340034003400340034003400340034EC
:10146000003400340034003400340034FF340034DD
:1014700000340034003400340034003400340034CC
:1014800000340034003400340034003400340034BC
:1014900000340034003400340034003400340034AC
:1014A0000034003400340034003400340034FF349D
:1014B000003400340034003400340034003400348C
:1014C000003400340034003400340034003400347C
:1014D000003400340034003400340034003400346C
:1014E000003400340034003400340034003400345C
:1014F000FF3400340034003400340034003400344D
:10150000003400340034003400340034003400343B
:10151000003400340034003400340034003400342B
:10152000003400340034003400340034003400341B
:101530000034FF340034003400340034003400340C
:1015400000340034003400340034003400340034FB
:1015500000340034003400340034003400340034EB
:1015600000340034003400340034003400340034DB
:1015700000340034FF3400340034003400340034CC
:1015800000340034003400340034003400340034BB
:1015900000340034003400340034003400340034AB
:1015A000003400340034003400340034003400349B
:1015B000003400340034FF3400340034003400348C
:1015C000003400340034003400340034003400347B
:1015D000003400340034003400340034003400346B
:1015E000003400340034003400340034003400345B
:1015F0000034003400340034FF340034003400344C
:10160000003400340034003400340034003400343A
:10161000003400340034003400340034003400342A
:10162000003400340034003400340034003400341A
:1016300000340034003400340034FF34003400340B
:1016400000340034003400340034003400340034FA
:1016500000340034003400340034003400340034EA
:1016600000340034003400340034003400340034DA
:10167000003400340034003400340034FF340034CB
:1016800000340034003400340034003400340034BA
:1016900000340034003400340034003400340034AA
:1016A000003400340034003400340034003400349A
:1016B0000034003400340034003400340034FF348B
:1016C000003400340034003400340034003400347A
:1016D000003400340034003400340034003400346A
:1016E000003400340034003400340034003400345A
:1016F000003400340034003400340034003400344A
:10170000FF3400340034003400340034003400343A
:101710000034003400340034003400340034003429
:101720000034003400340034003400340034003419
:101730000034003400340034003400340034003409
:101740000034FF34003400340034003400340034FA
:1017500000340034003400340034003400340034E9
:1017600000340034003400340034003400340034D9
:1017700000340034003400340034003400340034C9
:1017800000340034FF3400340034003400340034BA
:1017900000340034003400340034003400340034A9
:1017A0000034003400340034003400340034003499
:1017B0000034003400340034003400340034003489
:1017C000003400340034FF3400340034003400347A
:1017D0000034003400340034003400340034003469
:1017E0000034003400340034003400340034003459
:1017F0000034003400340034003400340034003449
:101800000034003400340034FF3400340034003439
:101810000034003400340034003400340034003428
:101820000034003400340034003400340034003418
:101830000034003400340034003400340034003408
:1018400000340034003400340034FF3400340034F9
:1018500000340034003400340034003400340034E8
:1018600000340034003400340034003400340034D8
:1018700000340034003400340034003400340034C8
:10188000003400340034003400340034FF340034B9
:1018900000340034003400340034003400340034A8
:1018A0000034003400340034003400340034003498
:1018B0000034003400340034003400340034003488
:1018C0000034003400340034003400340034FF3479
:1018D0000134013401340134013401340134013460
:1018E0000134013401340134013401340134013450
:1018F0000034003400340034003400340034003448
:101900000034003400340034003400340034003437
:101CD0001A340F341034FF3400340034003400342C
:101CE0000034003400340034003400340034003454
:101CF000FF34FF34FF340034003400340034003447
:101D0000FF34FF34FF34FF34003400340034003437
:101D1000003400340034FF34FF3400340034003425
:101D20000034003400340034003400340034003413
:101D30000034FF34FF340034003400340034003405
:101D40000034FF34FF34FF34FF34003400340034F7
:101D5000003400340034FF34FF34FF3400340034E6
:101D600000340034003400340034003400340034D3
:101D700000340034FF3400340034003400340034C4
:101D800000340034FF34FF34FF34FF3400340034B7
:101D9000003400340034FF34FF34FF34FF340034A7
:101DA0000034003400340034003400340034003493
:101DB0000034003400340034003400340034003483
:101DC000003400340034FF34FF34FF34FF34003477
:101DD0000034003400340034FF34FF34FF34FF3467
:101DE0000034003400340034003400340034003453
:101DF0000034003400340034003400340034003443
:101E00000034003400340034FF34FF34FF34FF3436
:101E100000340034003400340034FF34FF34FF3425
:101E2000FF34003400340034003400340034003413
:101E30000034003400340034003400340034003402
:101E400000340034003400340034FF34FF34FF34F5
:101E5000FF3400340034003400340034FF34FF34E5
:101E6000FF34FF34003400340034003400340034D4
:101E700000340034003400340034003400340034C2
:101E8000003400340034003400340034FF34FF34B4
:101E9000FF34FF3400340034003400340034FF34A5
:101EA000FF34FF34FF340034003400340034003495
:101EB0000034003400340034003400340034003482
:101EC0000034003400340034003400340034FF3473
:101ED000FF34FF34FF340034003400340034003465
:101EE000FF34FF34FF34FF34003400340034003456
:101EF000003400340034FF34003400340034003443
:101F00000034003400340034003400340034003431
:101F1000FF34FF34FF340034003400340034003424
:101F20000034FF34FF34FF34FF3400340034003415
:101F3000003400340034FF34FF3400340034003403
:101F400000340034003400340034003400340034F1
:101F50000034FF34FF3400340034003400340034E3
:101F600000340034FF34FF34FF34FF3400340034D5
:101F7000003400340034FF34FF34FF3400340034C4
:101F800000340034003400340034003400340034B1
:101F900000340034FF3400340034003400340034A2
:101FA000003400340034FF34FF34FF34FF34003495
:101FB000003400340034FF34FF34FF34FF34003485
:101FC0000034003400340034003400340034003471
:101FD0000034003400340034003400340034003461
:101FE0000034003400340034FF34FF34FF34FF3455
:101FF0000034003400340034FF34FF34FF34FF3445
:102000000034003400340034003400340034003430
:102010000034003400340034003400340034003420
:1020200000340034003400340034FF34FF34FF3413
:10203000FF340034003400340034FF34FF34FF3404
:10204000FF340034003400340034003400340034F1
:1020500000340034003400340034003400340034E0
:10206000003400340034003400340034FF34FF34D2
:10207000FF34FF340034003400340034FF34FF34C4
:10208000FF34FF34003400340034003400340034B2
:1020900000340034003400340034003400340034A0
:1020A0000034003400340034003400340034FF3491
:1020B000FF34FF34FF340034003400340034FF3484
:1020C000FF34FF34FF340034003400340034003473
:1020D000003400340034163440340234AA34AA34B4
:1020E000AA34AA34AA34AA34AA34AA34AA34AA3400
:1020F000AA34AA34AA34AA34AA34AA34553455349A
:102100005534553455345534553455345534553487
:102110005534553455345534553455345534553477
:102120005534553455345534553455345534553467
:10213000553455345534553455345534AA34AA34AD
:10214000AA34AA34AA34AA34AA34AA34AA34AA349F
:10215000AA34AA34AA34AA34AA34AA34163440348D
:1021600005340034003400340034003400340034CA
:1021700000340034003400340034003400340034BF
:1021800000340034003400340034003418343C345B
:102190001E343C341834003400340034003400342D
:1021A000003400340034003400340034003400348F
:1021B000003400340034003400340034003400347F
:1021C0000034003400340034003438347C347E343D
:1021D0003F343F347E347C343834003400340034AF
:1021E000003400340034003400340034003400344F
:1021F000003400340034003400340034003400343F
:102200000034003418343C341E343C341834003468
:10221000003400340034003400340034003400341E
:10222000003400340034003400340034003400340E
:1022300000340034003400340034003400340034FE
:10224000003438347C347E343F343F347E347C3444
:102250003834003418343C341E343C3418340034E0
:1022600000340034003400340034003400340034CE
:1022700000340034003400340034003400340034BE
:1022800000340034003400340034003400340034AE
:10229000003438347C347E343F343F347E347C34F4
:1022A00038341634403404340034003400340034FC
:1022B000003400340034003400340034003400347E
:1022C0000034003400340034FF34813481348134EC
:1022D0008134813481348134813481348134813456
:1022E000813481348134FF340034003400340034CC
:1022F000003400340034003400340034003400343E
:10230000003400340034003400347E34423442342B
:10231000423442344234423442344234423442340D
:10232000423442347E34003400340034003400340B
:1023300000340034003400340034003400340034FD
:102340000034003400340034003400343C3424348D
:1023500024342434243424342434243424342434BD
:1023600024343C340034003400340034003400346D
:1023700000340034003400340034003400340034BD
:102380000034003400340034003400340034183495
:1023900018341834183418341834183418341834DD
:1023A0001834003400340034163440340834803497
:1023B000803440342034103410342034403480349D
:1023C0008034403420341034103420344034083405
:1023D000083404340234013401340234043408343F
:1023E00008340434023401340134023404344034F7
:1023F000803480344034203410341034203440345D
:102400008034803440342034103410342034083484
:1024100004340234013401340234043408340834FE
:1024200004340234013401340234043408342034D6
:10243000403480348034403420341034103420341C
:102440004034803480344034203410341034043428
:1024500002340134013402340434083408340434BE
:1024600002340134013402340434083408341034A2
:1024700020344034803480344034203410341034DC
:1024800020344034803480344034203410340234DA
:10249000013401340234043408340834043402347E
:1024A0000134013402340434083408340434103460
:1024B000103420344034803480344034203410349C
:1024C000103420344034803480344034203401349B
:1024D000013402340434083408340434023401343E
:1024E000013402340434083408340434023420340F
:1024F000103410342034403480348034403420345C
:10250000103410342034403480348034403401346A
:1025100002340434083408340434023401340134FD
:1025200002340434083408340434023401344034AE
:10253000203410341034203440348034803440341B
:102540002034103410342034403480344034023489
:1025500004340834083404340234013401340234BD
:10256000043408340834043402340134023480342E
:1025700040342034103410342034403480348034DB
:102580004034203410341034203440348034043447
:10259000083408340434023401340134023404347D
:1025A000083408340434023401340134023416345B
:1025B000403404348034C034E034F0340F34073411
:1025C000033401348034C034E034F0340F34073441
:1025D0000334013400340034003400340034003457
:1025E000003400340034003400340034003400344B
:1025F0000034003408340C340E340F34F034E0343A
:10260000C034803408340C340E340F34F034E034E9
:10261000C0348034003400340034003400340034DA
:10262000003400340034003400340034003400340A
:10263000003400340F340E340C3408341034303489
:102640007034F0340F340E340C3408341034303419
:102650007034F0340034003400340034003400347A
:1026600000340034003400340034003400340034CA
:1026700000340034F03470343034103408340C3406
:102680000E340F34F03470343034103408340C34D9
:102690000E340F340034003400340034003400347D
:1026A000003400340034003400340034003400348A
:1026B000003400341634403408340034003400341C
:1026C000FF3400340034003400340034003400346B
:1026D0000034FF340034003400340034003400345B
:1026E000003400340034003418341834003400341A
:1026F0000034003400340034003400340034FF343B
:102700000034003400340034003400340034003429
:1027100000340034FF34003400340034003400341A
:102720000034003400341834243424341834003491
:10273000003400340034003400340034FF340034FA
:1027400000340034003400340034003400340034E9
:10275000003400340034FF340034003400340034DA
:10276000003400343C3442344234423442343C3449
:1027700000340034003400340034FF3400340034BA
:1027800000340034003400340034003400340034A9
:102790000034003400340034FF340034003400349A
:1027A00000347E3481348134813481348134813405
:1027B0007E340034003400340034003400340034FB
:1027C0000034003400340034183418340034003439
:1027D0000034003400340034003400340034003459
:1027E000FF3400340034003400340034003400344A
:1027F0000034FF340034003400340034003400343A
:1028000000340034003418342434243418340034B0
:102810000034003400340034003400340034FF3419
:102820000034003400340034003400340034003408
:1028300000340034FF3400340034003400340034F9
:10284000003400343C3442344234423442343C3468
:10285000003400340034003400340034FF340034D9
:1028600000340034003400340034003400340034C8
:10287000003400340034FF340034003400340034B9
:1028800000347E3481348134813481348134813424
:102890007E340034003400340034FF34003400341B
:1028A0000034003400340034003400340034003488
:1028B0000034003400340034FF3416344034123411
:1028C000063406347E3420341034003406340634A2
:1028D0007E342034103400340034003400340034AA
:1028E000003400340034003400340034063406343C
:1028F0007E34203410340034063406347E342034E0
:102900000C34FC34403420340034033403343F347A
:1029100010340834003400340034003400340034FF
:1029200000340034003400340034033403343F34C2
:102930001034083400340C340C34FC34403420346B
:102940007E34203410340034063406347E3420348F
:1029500010340034003400340034003400340034C7
:102960000034003400340034063406347E3420341D
:1029700010340034063406347E34203410340034ED
:10298000403420340034033403343F3410340834EA
:102990000034003400340034003400340034033494
:1029A000003400340034033403343F34103408342A
:1029B00000340C340C34FC34403420340034003403
:1029C00010340034063406347E342034103400349D
:1029D000003400340034003400340034063406344B
:1029E00000340034063406347E342034103400348D
:1029F000063406347E34203410340034003400347D
:102A00000034033403343F341034083400340034C9
:102A100000340034003400340034033403343F34D1
:102A20000034033403343F341034083400340C349D
:102A30000C34FC344034203400340034003400348E
:102A4000063406347E34203410340034003400342C
:102A50000034003400340034063406347E3420342C
:102A6000063406347E342034103400340634063400
:102A70007E34203410340034003400340034003408
:102A80000C34FC344034203400340034003400343E
:102A90000034003400340C340C34FC344034203422
:102AA0000C34FC34403420340034033403343F34D9
:102AB000103408340034003400340034003400345E
:102AC0007E342034103400340034003400340034B8
:102AD00000340034063406347E342034103400349C
:102AE0007E34203410340034063406347E342034EE
:102AF0001034003400340034003400340034003426
:102B000040342034003400340034003400340034C5
:102B100000340C340C34FC3440342034003403349E
:102B2000403420340034033403343F341034083448
:102B300000340034003400340034003400340334F2
:102B400010340034003400340034003400340034D5
:102B5000063406347E34203410340034063406340F
:102B600010340034063406347E34203410340034FB
:102B700000340034003400340034003406340634A9
:102B800000340034003400340034003400340C3499
:102B90000C34FC34403420340034033403343F34E8
:102BA0000034033403343F34103408340034003428
:102BB00000340034003400340034033403343F3430
:102BC0000034003400340034003400340634063459
:102BD0007E34203410340034063406347E342034FD
:102BE000063406347E34203410340034003400348B
:102BF0000034003400340034063406347E3420348B
:102C000000340034003400340034033403343F34DF
:102C10001034083400340C340C34FC344034203488
:102C20000C34FC344034203400340034003400349C
:102C30000034003400340C340C34FC344034203480
:102C40000034003400340034063406347E3420343A
:102C500010340034063406347E342034103400340A
:102C60007E34203410340034003400340034003416
:102C700000340034063406347E34203410340034FA
:102C8000003400340034033403343F341034083447
:102C900000340C340C34FC34403420340034003420
:102CA0004034203400340034003400340034003424
:102CB00000340C340C34FC344034203400340334FD
:102CC00000340034063406347E34203410340034AA
:102CD000063406347E34203410340034003400349A
:102CE0001034003400340034003400340034003434
:102CF000063406347E34203410340034063406346E
:102D00000034033403343F341034083400340C34BA
:102D10000C34FC34403420340034003400340034AB
:102D200000340034003400340034003400340C34F7
:102D30000C34FC34403420340034033403343F3446
:102D400016341F34033401340134073407340F348C
:102D50000F347F347F340F340F341F341F34073463
:102D600007340334033401340134043404340834A4
:102D700008344034403408340834103410340434F7
:102D80000434023402340F340F34033403343F3438
:102D90003F34FF34FF341F341F34073407340F34FB
:102DA0000F343F343F3408340834023402342034C2
:102DB0002034803480341034103404340434083423
:102DC000083420342034033403340F340F341F34D8
:102DD0001F34FF34FF340F340F34073407341F34EB
:102DE0001F340F340F3402340234083408341034E2
:102DF00010348034803408340834043404341034FB
:102E000010340834083419340F3444340134203475
:102E1000203420342034413443344B3420342034A3
:102E2000203420342034053420342034203420341D
:102E3000413443344B342034203420342034203483
:102E400004342034203420342034413443344B348F
:102E500020342034203420342034013420342034F1
:102E600020342034203420342034203420342034C2
:102E7000203420344E3441344B3420342034203438
:102E800020342034203420342034203420342034A2
:102E90002034203401340034003400340034003451
:102EA0000134F23400340034003400340334E034AC
:102EB0000034E0340034003405342834FE3428343F
:102EC000FE342834053424345434FE345434483425
:102ED0000534C434C83410342634463405346C34D4
:102EE0009234AA3484340A34033438344434823477
:102EF000003400340234A034C034003400340034D0
:102F000003348234443438340034003405342834F3
:102F100010347C34103428340534103410347C34AC
:102F200010341034023405340634003400340034D4
:102F30000534103410341034103410340234063494
:102F400006340034003400340534043408341034BA
:102F50002034403404347C34823482347C34003471
:102F600003344234FE340234003400340434463432
:102F70008A349234623400340434443482349234D7
:102F80006C3400340534183428344834FE340834A2
:102F90000434E434A234A2349C34003404343C3489
:102FA000523492340C340034043480348E349034EF
:102FB000E034003404346C34923492346C34003491
:102FC00004346034923492347C3400340234363425
:102FD00036340034003400340234353436340034AE
:102FE000003400340434103428344434823400343F
:102FF00005342834283428342834283404348234DE
:1030000044342834103400340534403480348A3455
:103010009034603405344C3492349E3482347C34A1
:1030200005343E344834883448343E340534FE3464
:103030009234923492346C3405347C348234823449
:10304000823444340534FE348234823482347C3415
:103050000534FE3492349234923492340534FE3482
:10306000903490349034903405347C3482349234EB
:1030700092345C340534FE34103410341034FE3491
:1030800003348234FE348234003400340434043493
:1030900002340234FC3400340534FE341034283455
:1030A000443482340534FE340234023402340234AF
:1030B0000534FE34403430344034FE340534FE34BC
:1030C000403420341034FE3405347C34823482346D
:1030D00082347C340534FE3490349034903460343F
:1030E00005347C3482348A3484347A340534FE34B2
:1030F0009034983494346234053464349234923485
:1031000092344C34053480348034FE34803480343E
:103110000534FC34023402340234FC340534F8340F
:10312000043402340434F8340534FC3402341C34DE
:103130000234FC340534C634283410342834C63400
:103140000534E03410340E341034E0340534863461
:103150008A349234A234C2340334FE34823482344A
:10316000003400340534403420341034083404343E
:10317000033482348234FE34003400340534203485
:103180004034803440342034053401340134013477
:10319000013401340234C034A0340034003400342B
:1031A000043404342A342A341E3400340434FE3403
:1031B000223422341C34003404341C3422342234AB
:1031C0002234003404341C3422342234FE340034DB
:1031D00004341C342A342A341834003404341034AF
:1031E0007E3490344034003404341834253425348B
:1031F0003E3400340434FE34103420341E340034A1
:1032000003342234BE340234003400340434023433
:1032100001342134BE3400340434FE340834143410
:103220002234003403348234FE3402340034003457
:1032300005341E342034183420341E3404343E3413
:10324000103420341E34003404341C34223422342C
:103250001C34003404343F3424342434183400340F
:1032600004341834243424343F34003404343E34D9
:103270001034203420340034043410342A342A34F6
:1032800004340034033420347E34203400340034D9
:1032900004343C34023402343C34003405343834D1
:1032A000043402340434383405343C3402340C34ED
:1032B00002343C34053422341434083414342234B7
:1032C00005343834053405343E34003404342634AF
:1032D0002A34323400340034033410346C348234F1
:1032E000003400340134FF3400340034003400343E
:1032F000033482346C341034003400340434003429
:103300003E343E343E3480340434773441346334C4
:103310004134F734043414342234143422349434D1
:02400E00C428C4
:02401000FF3E71
:04420000FF00013486
:00000001FF
